:100000005D280F39A0000310A00DA00D1F08E039D6
:10001000200401389F000030A100323025209F14B9
:100020009F1810281E08A10083161E085828A30137
:10003000A200FF30A207031CA307031C58280330AB
:10004000A100E33025201928A101F43EA000A10958
:10005000FE30031C2E28A00703182B28A0076400DD
:10006000A10F2B2800002018352820183728080059
:10007000A20002304128A20001304128A20006302F
:100080004128A80023082102031D48282208200235
:10009000043003180130031902302805031DFF3016
:1000A00058280038031DFF300405031DFF30582871
:1000B00083130313831264000800831690018312D4
:1000C00083309F00831603309F008312073099000E
:1000D00083160B30850083128501831677308F00DD
:1000E00083129501831605153230831217209A204A
:1000F0004608B8004708B9003230B8070318B90AF3
:10010000C001C101C001C1014008A0004108A10017
:100110000130A3002C303B20031D992883160515C0
:1001200083129A20B020A520BC20C00A0319C10F59
:100130008428802883160515003083120120C6000C
:100140002108C7005030172008008316051501301C
:1001500083120120C8002108C90050301720080070
:100160004608A0004708A1003908A30038083E202F
:10017000031DBB28152108004808A0004908A1005C
:100180000330A300E8303B20C2004008A000410833
:10019000A1000130A3002B303820C40042088400A5
:1001A00044085120C400C5006400440845040319F4
:1001B000DA2827214808A0004908A1000330A3003D
:1001C000E8303B20C2004008A0004108A100A30184
:1001D000C8303820C4004208840044085120C400BC
:1001E000C5006400440845040319F728392148086C
:1001F000A0004908A1000330A300E8303B20C20062
:100200004008A0004108A100A30164303820C400C8
:100210004208840044085120C400C500640044081A
:100220004504031914294B210800851283168512F1
:100230008312051283160512051183120511831608
:10024000051183121730A300D430182008000512BE
:1002500083160512831285168316851205118312E3
:1002600005118316051183121730A3007030182072
:10027000080005168316051283128512831685124F
:100280000511831205118316051183121730A3007F
:100290007030182008000516831605128312851683
:1002A0008316851205118312051183160511831219
:0E02B0001730A30070301820080063005D298D
:02400E00F43C80
:00000001FF
